:100000000C94B4020C94EC020C94EC020C94EC02F0
:100010000C94EC020C94EC020C94EC020C94EC02A8
:100020000C94EC020C94EC020C94E7250C94B92689
:100030000C94C6200C94EC020C94EC020C94EC0290
:100040000C94EC020C94EC020C94EC020C94EC0278
:100050000C94EC020C944E210C94EC020C94EC02E7
:100060000C94EC020C94EC020C94EC020C94EC0258
:100070000C94EC020C94EC020C94EC020C94EC0248
:100080000C94EC020C94EC020C94EC020C94EC0238
:100090000C94EC020C94EC020C94EC020C94EC0228
:1000A0000C94EC020C94EC020C94EC022E052E0540
:1000B0005A055A05C205E005F806F806EB05840660
:1000C0009506950626274D2745284D27452899272B
:1000D000BC27452813282228290014001A000800EC
:1000E000150017001C0018000C00120013002B0054
:1000F00004001600070009000A000B000D000E00A6
:100100000F002800E1001D001B000600190005007B
:100110001100100036003700A800E2000151000075
:100120002C00000000002A0000000251E000000046
:1001300001001E001F0020002100220023002400D7
:100140002500260027002D002E00350001000100AB
:10015000010001000100010034003300E100500003
:1001600051004F0001000100010001003800310082
:1001700001000100010000000100000000004C002F
:10018000000001000100000053003A003B003C0069
:100190003D003E003F00400041004200430044005B
:1001A00045005200010001000100010001000100B2
:1001B0002F003000E100500051004F0057005A005E
:1001C00062005900010001000100C35CC85C00002E
:1001D000C65C00000000CA5C00000100C45C0000B6
:1001E00000047F3F1F643214643214783C1E1E14D6
:1001F0000A052223252628292A2C2D2F3032333593
:1002000036383A3B3D3E4042434547494A4C4E50C2
:1002100051535557595A5C5E6062646668696B6DEC
:100220006F71737577797B7D7F81838587898A8CF0
:100230008E90929496989A9C9E9FA1A3A5A7A8AAF7
:10024000ACAEAFB1B3B4B6B8B9BBBCBEBFC1C2C32C
:10025000C5C6C7C9CACBCCCDCED0D1D2D2D3D4D5C6
:10026000D6D7D7D8D9D9DADADBDBDBDCDCDCDCDCEF
:10027000DDDDDDDDDCDCDCDCDCDBDBDBDADAD9D9C7
:10028000D8D7D7D6D5D4D3D2D2D1D0CECDCCCBCA55
:10029000C9C7C6C5C3C2C1BFBEBCBBB9B8B6B4B37B
:1002A000B1AFAEACAAA8A7A5A3A19F9E9C9A989611
:1002B0009492908E8C8A89878583817F7D7B7977E4
:1002C0007573716F6D6B6968666462605E5C5A59C4
:1002D00057555351504E4C4A4947454342403E3D85
:1002E0003B3A3836353332302F2D2C2A2928262513
:1002F0002322FFAA7F5540000101010101010101F4
:1003000001020202020202020202030303030303C8
:100310000303040404040404040505050505060696
:100320000606060707070707080808080909090954
:100330000A0A0A0B0B0B0C0C0C0D0D0D0E0E0E0FFA
:100340000F0F10101111111212131314141515168A
:10035000161717181819191A1A1B1B1C1D1D1E1EFB
:100360001F2020212222232424252626272829294C
:100370002A2B2C2D2D2E2F30313232333435363777
:1003800038393A3B3C3D3E3F404142434445464775
:1003900048494A4C4D4E4F50515354555658595A4E
:1003A0005B5D5E5F616264656668696B6C6D6F70F2
:1003B00072737577787A7B7D7E8082838587888A61
:1003C0008C8E8F91939596989A9C9EA0A2A3A5A798
:1003D000A9ABADAFB1B3B5B7BABCBEC0C2C4C6C994
:1003E000CBCDCFD1D4D6D8DBDDDFE2E4E7E9EBEE4D
:1003F000F0F3F5F8FAFDFF0E034B0061007200699F
:10040000006E006100000018034D00690073006F6A
:10041000006E006F0057006F0072006B00730000E9
:10042000000403090409023B00020100A0FA0904C8
:100430000000010301010009211101000122400017
:100440000705810308000109040100010300000001
:1004500009211101000122B60007058203200001D5
:100460001201000200000008EDFE56C40100010266
:10047000000105010902A10185020901A100050988
:10048000190129081500250195087501810205014A
:10049000093009311581257F9502750881060938D3
:1004A0001581257F950175088106050C0A3802150E
:1004B00081257F950175088106C0C005010980A1CD
:1004C00001850319012AB700150126B700950175AA
:1004D000108100C0050C0901A101850419012AA0A1
:1004E00002150126A002950175108100C0050109C1
:1004F00006A1018506050719E029E71500250195E4
:1005000008750181020507190029EF1500250195DD
:10051000F0750181020508190129059505750191FC
:1005200002950175039101C005010906A1010507A6
:1005300019E029E71500250195087501810295014B
:10054000750881010507190029FF150026FF009590
:1005500006750881000508190129059505750191A1
:1005600002950175039101C011241FBECFEFDAE09F
:10057000DEBFCDBF04B603FE18C080915C0390912E
:100580005D03A0915E03B0915F038730904BA7405D
:10059000B04B59F410925C0310925D0310925E030D
:1005A00010925F03E0E0F8E3099511E0A0E0B1E00C
:1005B000E0EFF2E502C005900D92A03FB107D9F738
:1005C00023E0A0EFB1E001C01D92AC35B207E1F726
:1005D0000E9429130C9476290C940000811106C006
:1005E000662311F08BE409C08EE407C0813039F432
:1005F000662311F089EA01C08AEA0E94DC0481E0E6
:10060000089581E0089581E008950C94030308950E
:100610000C9407031F93CF93DF9300D000D01F9259
:10062000CDB7DEB749835A836B833091F30189815B
:100630009A81311114C0662359F0222349F00E9497
:100640003509182F682F89819A810E94DE0803C01E
:100650000E940909182F69817A81812F04C00E94A4
:10066000350969817A810F900F900F900F900F904C
:10067000DF91CF911F910C949410FC01262F4081A3
:1006800051816281738184810C940A0381E0089511
:10069000CF93DF93EC0160E00E943D03BE01DF9148
:1006A000CF910C9408030C94DA110C94D611089590
:1006B0000E9488070E9457032FEF84E39CE021509B
:1006C00080409040E1F700C000000C9474210F932B
:1006D0001F93CF93DF938C0161E00E943D03EC01F7
:1006E000B8010E940503882309F444C0B801CE0173
:1006F0000E94111F8823F1F1B801CE010E942C1C29
:100700008823C1F1B801CE010E946D1E882391F1AA
:10071000B801CE010E94321B882361F1F801828169
:10072000882309F1CB358DE5D807C1F050F4C11508
:10073000FCE5DF0781F0CF3DDC45A9F40E946C0E9B
:1007400019C0CC35EDE5DE0761F0CD35DD4559F456
:100750000E94AF0D08C00E9458030CC00E94B80D43
:1007600002C00E94BB0DC801DF91CF911F910F9174
:100770000C94010380E0DF91CF911F910F910895B8
:100780000E94A8200C94D9030E94DC030C94AE2094
:1007900008950C94C80381E008950C94CB03089548
:1007A000CF93C82F0E94C9038C2F0E94CD03CF91F5
:1007B000089580E00C94D0030E946D1F0C94D00328
:1007C0000E946D1F9091F201891721F08093F20130
:1007D0000C94D0030895CF93DF93CDB7DEB72B975A
:1007E0000FB6F894DEBF0FBECDBF4F835887698721
:1007F0007A878B8761110E94FB0C9E012F5F3F4F10
:1008000086E0F90111928A95E9F785E0FE013796B5
:10081000D90101900D928A95E1F789819A814C81E5
:100820005D81452B31F09F3F31F491E08F3F19F40A
:1008300003C091E001C090E090FF09C049815A8156
:100840006B817C818D819E810E941C0C05C0C90139
:100850000E9446038111F2CF2B960FB6F894DEBFAB
:100860000FBECDBFDF91CF910895FC0180819181B2
:100870000E9477090895CF93882309F450C0C82FA8
:100880008CEF8C0F813AD0F46C2F80910201909103
:1008900003010E94E31F882349F06C2F809102011D
:1008A000909103010E946E200E941D0D6C2F80917B
:1008B0000201909103010E9463200CC080E28C0F22
:1008C000883058F4C77081E001C0880FCA95EAF7F4
:1008D0000E94DE0CCF910C941D0DEBE5EC0FE33084
:1008E00040F4F0E0ED58FE4F808190E0CF910C9401
:1008F000A11FE8E5EC0FE73150F4F0E0EE0FFF1F29
:10090000EB5BFE4F80819181CF910C94B71FCD3E60
:1009100030F08C2F0E94AD13CF910C945714CF91CF
:100920000895882389F19CEF980F913A40F4682F3D
:1009300080910201909103010E946E200DC090E20F
:10094000980F983058F4877091E001C0990F8A95FC
:10095000EAF7892F0E94E40C0C941D0D9BE5980F7B
:10096000933020F480E090E00C94A11F98E5980F5C
:10097000973120F480E090E00C94B71F8D3E20F07A
:100980000E9404140C94571408951F93CF93DF937F
:10099000182FEB010E943B04209741F08FE99FE064
:1009A0000197F1F700C000002197F6CF812FDF916A
:1009B000CF911F910C949104893319F060E070E09D
:1009C00002C060E570E00C94C504882321F00E9409
:1009D000DE0C0C941D0D0895882321F00E94E40C78
:1009E0000C941D0D0895CF92DF92EF92FF920F931A
:1009F0001F93CF93DF937C01D62FC72FFC01128169
:100A0000058102950F700E94D40C8823B9F0112340
:100A1000A9F08C2F807F803421F080E28D0F883008
:100A200068F08091FC0282FD09C082E00E947D0D89
:100A30000E94D40C91E0D82ED92601C0D12CCC2E06
:100A4000C2948FE0C8228C2D90E08C30910508F084
:100A5000CFC1FC01EA5AFF4F0C94D1288C2F807F24
:100A6000CF70882311F0C295C07F112399F0CC2359
:100A700009F4AAC180E28D0F883010F0D11104C0B2
:100A80008C2F0E94DE0C03C08C2F0E94EE0C0E9463
:100A90001D0D9AC18D2F0E949104CC2309F4A8C189
:100AA00080E28D0F883038F1DD2329F18C2F0E94F0
:100AB000F40C24C08C2F807FCF70803211F0C2954F
:100AC000C07FDD2319F0D130A1F13DC08091FC023F
:100AD00082FF17C0112349F0CC2329F08C2F0E94EC
:100AE000DE0C0E941D0D80E070C180E00E94910428
:100AF000CC2309F47DC18C2F0E94E40C0E941D0DB3
:100B000077C1112371F0002341F0013031F40E94CC
:100B1000FE0C8C2B0E94060D6BC10E94FE0C8C2BD0
:100B20001DC0002319F0013009F462C10E94130DA9
:100B300025C0112321F0063008F05AC10EC005303F
:100B400008F056C11BC0112361F0002331F0F701FA
:100B5000858180FF39C18F7085838C2F0E94E504C9
:100B600047C1002359F0D93309F03FC1FFEF07EE29
:100B700013E0F15000401040E1F735C18C2F0E9486
:100B8000EC0436C18C2F86958695837019F08130E0
:100B900061F02EC1112321F08D2F9C2F937002C084
:100BA00080E090E00E94A11F2BC1112321F08D2F26
:100BB0009C2F937002C080E090E00E94B71F20C17C
:100BC0008D2F112319F00E94AD1302C00E9404144E
:100BD0000E94571415C18C2F837009F047C0111162
:100BE0000BC12D2F229526952770220F220F6D2FD6
:100BF0006F70862F90E0A0E0B0E0022E04C0880F56
:100C0000991FAA1FBB1F0A94D2F7D4FF10C04FE050
:100C100050E060E070E004C0440F551F661F771F6E
:100C20002A95D2F7409550956095709503C040E0A5
:100C300050E0BA01C695C695C3708A019B01082B86
:100C4000192B2A2B3B2BC901B801C23049F058F4AB
:100C5000C13019F00E94F407CFC00E94E207CCC057
:100C60000E940608C9C00E94E007C6C0112319F0FF
:100C70008C2F817001C08695882309F4BDC02D2F6B
:100C8000229526952770220F220F6D2F6F70862FC9
:100C900090E0A0E0B0E0022E04C0880F991FAA1FC8
:100CA000BB1F0A94D2F7D4FF10C04FE050E060E0C1
:100CB00070E004C0440F551F661F771F2A95D2F7B6
:100CC000409550956095709503C040E050E0BA01A2
:100CD000C695C695C3708A019B01082B192B2A2B38
:100CE0003B2BC901B801C23049F058F4C13019F0AA
:100CF0000E94B90881C00E94A7087EC00E94CB084C
:100D00007BC00E941A0878C0CF70112339F08C2F55
:100D10000E9440088D2F0E94E5046EC08D2F0E9416
:100D2000EC048C2F0E94610867C0D23F21F128F4A7
:100D3000D03F41F0D13FC1F043C0D33F19F1D43F80
:100D400079F03EC0112341F0053008F051C08C2FDE
:100D50008F710E9486084CC0063008F049C0F7CF5A
:100D60008091FC0282FF18C0112339F08C2F8F7103
:100D70000E9440083DC01123C9F38C2F8F710E943F
:100D8000610836C0112329F08C2F8F710E942B0827
:100D90002FC00E9426082CC0112349F0CF718C2F40
:100DA0000E94400863E08C2F0E94620D21C081E008
:100DB0000E947D0D0230E0F082E00E947D0D18C09F
:100DC000112331F0002391F28D2F0E943B0410C0BB
:100DD000002399F2D93349F41FEF27EE33E0115085
:100DE00020403040E1F700C000008D2F0E949104A8
:100DF00088EF8C0D843020F40E946D1F0E94D00378
:100E0000DD20C9F00E94D00C80FD15C0F7011282D0
:100E10000E94CA0C0E944008C7010E943C070E9421
:100E2000CA0CDF91CF911F910F91FF90EF90DF904F
:100E3000CF900C946108DF91CF911F910F91FF909B
:100E4000EF90DF90CF9008950F931F93CF93DF9390
:100E5000EC01688179818A810E9482098C010E945B
:100E6000DD080E94CE07B801CE010E94F304DF9195
:100E7000CF911F910F910895CF93DF93EC0198814B
:100E800089812B813C81232B31F08F3F31F481E02C
:100E90009F3F19F403C081E001C080E080FD1DC0C8
:100EA000CE010E946703811110C00E94D40C8823D8
:100EB000A1F08A81882389F08091FC0282FD0DC017
:100EC00082E0DF91CF910C947D0DCE010E9424072A
:100ED000CE01DF91CF910C944803DF91CF9108951B
:100EE00080E090E00E94A11F80E090E00E94B71F88
:100EF0000E94FB0C0E941D0D0E94F8140C945714C4
:100F000080910201909103010E9479200C94700756
:100F10000E94EB0C0C94800792959F70963079F0AC
:100F200010F4925001C09A50923068F4803F69F0FA
:100F300018F4883E40F409C0843F29F406C0883E76
:100F400020F0813F11F080E0089581E00895FC01D8
:100F5000808191810E9477090E948C070895CF9328
:100F6000DF9300D000D01F92CDB7DEB70F900F9067
:100F70000F900F900F90DF91CF910895CF93DF9353
:100F800000D000D000D0CDB7DEB726960FB6F894CB
:100F9000DEBF0FBECDBFDF91CF91089508950895B4
:100FA0000C94CF070C94D0070E94D20760931602CE
:100FB0007093170280931802909319020C94700793
:100FC0000C94D4070F931F930091160210911702EF
:100FD0002091180230911902602B712B822B932BD8
:100FE0001F910F910C94D4070F931F930091160239
:100FF0001091170220911802309119026023712379
:10100000822393231F910F910C94D4070F931F9366
:1010100000911602109117022091180230911902C6
:1010200060277127822793271F910F910C94D40773
:101030000C94CF070E941808609312027093130259
:1010400080931402909315020C94700760E070E096
:10105000CB010C941A080F931F9341E050E060E01D
:1010600070E08A019B0104C0000F111F221F331F73
:101070008A95D2F7C901B8011F910F910C941A08F3
:101080000F931F9341E050E060E070E004C0440F14
:10109000551F661F771F8A95D2F780911202909193
:1010A0001302A0911402B09115028A019B01082B32
:1010B000192B2A2B3B2BC901B8011F910F910C94BE
:1010C0001A080F931F9341E050E060E070E004C005
:1010D000440F551F661F771F8A95D2F7409550958C
:1010E000609570958091120290911302A091140264
:1010F000B09115028A019B01082319232A233B235F
:10110000C901B8011F910F910C941A080F931F93F6
:1011100041E050E060E070E004C0440F551F661FDE
:10112000771F8A95D2F78091120290911302A091B5
:101130001402B09115028A019B01082719272A275A
:101140003B27C901B8011F910F910C941A080F9306
:101150001F930091120210911302209114023091FA
:101160001502602B712B822B932B1F910F910C94E6
:101170001A080F931F9300911202109113022091ED
:1011800014023091150260237123822393231F914F
:101190000F910C941A080F931F9300911202109153
:1011A00013022091140230911502602771278227C3
:1011B00093271F910F910C941A0808952BE0929F8A
:1011C000800D1124E82FE695E695E695877051E0AD
:1011D00001C0550F8A95EAF785E0E89FF0011124D8
:1011E000EC50FE4F20E030E070E04081CB01022E59
:1011F00002C0969587950A94E2F7817081958427BD
:101200008523842781932F5F3F4F2530310569F770
:1012100008952BE0929F800D1124682F66956695A6
:101220006695982F977085E0689FB001112440E083
:1012300050E080E0FB01E40FF51FEC50FE4F2081F1
:1012400030E0092E02C0369527950A94E2F7217006
:101250003327042E01C0220F0A94EAF7822B4F5F36
:101260005F4F4530510531F70895BF92CF92DF921D
:10127000EF92FF920F931F93CF93DF938C01C09057
:101280001202D0901302E0901402F09015028091A7
:10129000160290911702A0911802B0911902C82A63
:1012A000D92AEA2AFB2ACFE1D0E0D701C6010C2EC9
:1012B00004C0B695A795979587950A94D2F780FDB7
:1012C00004C0219790F7B12C07C0BC2EB8018C2F19
:1012D0000E94A7100197A9F38B2DDF91CF911F9149
:1012E0000F91FF90EF90DF90CF90BF900895CF9334
:1012F000DF93EC010E943509BE010E94A710DF9127
:10130000CF9108951F93CF93DF93EB019091F30159
:10131000992321F0CB010E94770913C0882349F05B
:10132000CB010E943509182F682FCE010E94DE08DC
:1013300004C0CB010E940909182FBE01812F0E9411
:10134000A710DF91CF911F9108951F93CF93DF9343
:10135000C0911A0216E080911B02C81799F0D0E0E4
:101360001C9FF0011D9FF00D1124E45EFD4F408194
:10137000518162817381848195810E94BE0721968B
:10138000C770E9CFDF91CF911F91089540914C0232
:1013900050914D0260914E0270914F028091500227
:1013A000909151020C94BE07EF92FF920F931F93FE
:1013B000CF93DF938091510282958F7009F065C0C1
:1013C00080914E02882309F460C080911A02F09047
:1013D0001B0210914C0200914D0260914F027091DE
:1013E000500291E01F3F09F090E0C0910001D091C0
:1013F0000101292F96E0E92E8F1509F446C06115E9
:10140000710521F00F3F21F030E003C031E001C051
:10141000322F90E030FD36C0E89EF001E99EF00DDD
:101420001124DF01A45EBD4F11963C91119730133A
:1014300029C03C91311326C012963C91129731116C
:1014400021C013964D915C911497461B570B4C1776
:101450005D07C0F4809151028F70806180935102CA
:10146000EF5DFD4F80818F70806180838CE492E01E
:101470000E943C07DF91CF911F910F91FF90EF9059
:101480000C94A50901968770B7CFDF91CF911F917A
:101490000F91FF90EF9008959F92AF92BF92CF92DD
:1014A000DF92EF92FF920F931F93CF93DF93CDB70D
:1014B000DEB761970FB6F894DEBF0FBECDBF8C01CB
:1014C00085E0F801DE011D9601900D928A95E1F705
:1014D000D8011296EC9090914C02E0914D0220912F
:1014E0004F02309150022115310531F0EF3F31F4B8
:1014F00081E09F3F19F403C081E001C080E0B82F74
:10150000B1709B2E80FD47C1D8014C9111965C9122
:1015100011971396AD90BC9014978CE4C82E82E07E
:10152000D82EF0904E02B501621B730B2091000182
:1015300030910101FF2009F4D9C080915102621756
:10154000730708F095C0282F207F09F052C05E1362
:1015500013C0491311C0FE2CE1100EC08F708061C2
:10156000809351020E94C609C6010E943C078091E7
:101570005102F80185834DC1AB2831F05F3F31F452
:1015800081E04F3F19F403C081E001C080E080FD9D
:1015900003C081E08E2502C080E090E0F82FF1705A
:1015A000FF2E80FF1CC080911A0220911B0236E0A2
:1015B000821709F40BC190E0389FF001399FF00DBC
:1015C0001124E45EFD4F6181561306C0608146130D
:1015D00003C06281E61203C001968770E9CFFE2C3A
:1015E000EE2009F416C1809151028160809351026E
:1015F00054C05E1306C0491304C0E11002C0F801D4
:1016000099C0C8010E94A707882361F1EE2051F11B
:1016100020915102822F82958F7090E0029774F092
:1016200080914C0290914D0298878F831986BB86DA
:10163000AA862C87CE0107960E943C0786E0F80117
:10164000ACE4B2E001900D928A95E1F70E94D409D2
:101650000E94C6090AC05E1711F1C8010E94A707BF
:1016600081112CC0C8010E943C07FF24F394D1C013
:10167000282F207F81F77A2DB98AA88A6E2D898933
:101680000E94AF078CE492E00E943C0786E0D601FE
:101690001D928A95E9F70E94C609F12CBAC0491338
:1016A000DCCFE110DACFF8018583C8010E943C0746
:1016B00086E0D6011D928A95E9F7ABC0EE2091F243
:1016C00020915102822F82958F7090E002970CF446
:1016D000B5CF80914C0290914D029A8389831B82F1
:1016E000BD82AC822E83CE010196A6CF621773070E
:1016F00008F044C0FE2CEE2009F4B4CF5E1330C0D5
:1017000049132EC02091510220FD21C0822F8295C5
:101710008F70482F50E041155105C9F0F80125831D
:101720004F30510541F08F5F982F9295907F822F17
:101730008F70892B8583C8010E943C0786E0F801E1
:10174000ACE4B2E001900D928A95E1F73CC086E0EE
:10175000F801ACE4B2E001900D928A95E1F759C02E
:10176000C8010E94A707811169CF80915102816051
:1017700080935102C8010E943C074BC07A2DB98A60
:10178000A88A6E2D89890E94AF0786E0D6011D9236
:101790008A95E9F718C0EE2009F464CFC8010E94C9
:1017A000A707F82E882309F45DCF86E0F801ACE4A2
:1017B000B2E001900D928A95E1F78CE492E00E94EC
:1017C00035040E94D4090E94C60923C04D875E8754
:1017D0008D859E850E947709292F22952F702230B2
:1017E00028F49F7039F0811105C00BC0243028F413
:1017F0009F7049F4805E883020F0C8010E943C0749
:101800009F2CF92C06C0D80115969C91907F91F7DA
:10181000F8CF8F2D61960FB6F894DEBF0FBECDBF07
:10182000DF91CF911F910F91FF90EF90DF90CF90BC
:10183000BF90AF909F9008951F93CF93DF93CDB744
:10184000DEB72C970FB6F894DEBF0FBECDBF4F8327
:10185000588769877A878B879C87CE0107960E9475
:101860004C0A8823D1F09F8188852A853B85232BCC
:1018700031F08F3F31F481E09F3F19F403C081E0E4
:1018800001C080E080FD47C04F81588569857A8519
:101890008B859C850E94BE073EC086E0FE01379680
:1018A000DE01119601900D928A95E1F7FF81E8859E
:1018B0006A857B856115710531F0EF3F31F481E078
:1018C000FF3F19F403C081E001C080E080FD23C028
:1018D00020911B0230E0C901019687709927409141
:1018E0001A0250E084179507F1F1F983EA837D83AA
:1018F0006C8396E0929FD001939FB00D1124A45E5B
:10190000BD4FFE01319601900D929A95E1F78093BB
:101910001B020E94A50916E080911A0290911B02F9
:10192000891771F1189FC0011124845E9D4F0E9498
:101930004C0A882329F1E0911A021E9FF00111241C
:10194000E45EFD4F40815181628173818481958184
:101950000E94BE0780911A0290E001968770992735
:1019600080931A02D9CF0E94880710921B0210920E
:101970001A02ECE4F2E086E0DF011D928A95E9F7B5
:101980002C960FB6F894DEBF0FBECDBFDF91CF917E
:101990001F9108958091720285958595859508958A
:1019A000809172028770089590917202977081E021
:1019B00009F480E008958091950208959091950230
:1019C000892B8093950208958095909195028923A3
:1019D0008093950208951092950208959091940233
:1019E000892B809394020895809590919402892385
:1019F0008093940208951092940208958091730246
:101A0000089508950C94010D0C94020D9091FC0220
:101A100092FD08C090917302981721F08093730291
:101A20000C94040D089580917302882329F010927C
:101A3000730280E00C94040D0895CF93DF93E0913E
:101A40000201F0910301809195028083E0910201EF
:101A5000F0910301908180919402892B8083809181
:101A60007302882381F0E0910201F09103019081DB
:101A7000892B808380910201909103010E94CD1FE8
:101A800081110E94130DC0910201D091030140E227
:101A900050E062E572E0CE010E942129892B69F0B5
:101AA00080E2FE01A2E5B2E001900D928A95E1F795
:101AB000CE01DF91CF910C94791FDF91CF910895E2
:101AC0000C94010D9091FC0292FD10C098E0899F4A
:101AD00090011124262B209372020E9440088091CD
:101AE00072028595859585950C94600D0C9440083F
:101AF0001092720280E00C94600D20917202809529
:101B0000822380937202982F977099F430E0482FC7
:101B1000082E000C550B2417350759F09091FC0244
:101B200092FD07C08595859585950E9461080C9466
:101B3000780D08959091FC0292FB222720F9281736
:101B400069F080FB92F99093FC028091FB029091E6
:101B5000FC020E94E80D82E00C947D0D08958091B6
:101B6000FC0282FB882780F991E089270C949A0D6A
:101B700081E00C949A0D80E00C949A0D6FEF7FEF4A
:101B800080E090E00C94602980E090E00E943C2985
:101B900021E0893E9E4F09F020E0822F089582E0E7
:101BA00090E00C942E2983E090E00C942E29CF93A2
:101BB00084E090E00E942E29C82F82E290E00E94EB
:101BC0002E292C2F30E0A901582BCA01CF9108955E
:101BD000CF93C92F682F84E090E00E9442296C2F98
:101BE00082E290E0CF910C944229AB01BC018FE0DE
:101BF00090E00C945429AB01BC0183E190E00C947B
:101C0000542960E070E0CB010C94FB0D60E070E0C3
:101C1000CB010E94F50D0C94010E69EE7EEF80E081
:101C200090E00E94602960E082E090E00E944229FA
:101C300060E083E090E00E94422910921602109228
:101C40001702109218021092190260E084E090E0EE
:101C50000E94422960E082E290E00E94422960E016
:101C600085E090E00E94422960E086E090E00E94DA
:101C700042296FEF87E090E00E94422940E050E067
:101C8000BA0188E090E00E94542960E08DE090E085
:101C90000E94422940E050E0BA0188E190E00E94B1
:101CA000542960E087E190E00E94422940E050E042
:101CB000BA018CE190E00E94542960E070E080E27B
:101CC00090E00E94602940E050E0BA0188E190E095
:101CD0000E9454290C94060E0C940D0E682F8EE071
:101CE00090E00C9442290E9433216093A6027093E5
:101CF000A7028093A8029093A9026093A202709316
:101D0000A3028093A4029093A50208950E94332118
:101D10006093A6027093A7028093A8029093A902F1
:101D200060939E0270939F028093A0029093A10201
:101D3000089585B7806885BF85B7806885BF089599
:101D400081E008950C94A00E08950C94A40E0C94B8
:101D5000A40E0C94A70E0C94A40E0C94AB0E0C9431
:101D6000A40E0E94990E83E891E10E94631F0E94D5
:101D7000AF0E0C94AD0E0E94A50E0C94A40E0E9402
:101D80009D110C94CF030E941E210E9482120E947A
:101D9000BF0E0E94511A0E947D1DEBEFF2E0808180
:101DA000806880838091FB029091FC020E94E80D84
:101DB0000C94A90E5F926F927F928F929F92AF9236
:101DC000BF92CF92DF92EF92FF920F931F93CF9328
:101DD000DF93CDB7DEB72A970FB6F894DEBF0FBEFC
:101DE000CDBF0E949712C82E81110E94730E36E952
:101DF000832E32E0932E00E010E0502E802F0E94C0
:101E0000C1115C01F401619071904F01682679263F
:101E100061147104B1F40F5F1F4F0430110569F7AD
:101E20008FEF89838A831B820E9427218160782F0C
:101E30009D838C8349815A816B818D810E94EB0344
:101E40003AC08091AA0281FD0E94CA11D12CEE24D1
:101E5000E394F12CC3018E219F21892B29F10E944B
:101E6000A20E8823A9F0DE825F82AE20BF2081E02F
:101E7000AB2809F480E088870E9427218160782FB1
:101E80009A8789874E815F8168858A850E94EB03E6
:101E9000000F111FF801EA56FD4F80819181E8265D
:101EA000F926F182E08207C0D394EE0CFF1CFBE020
:101EB000DF12D0CFB0CF81E0C11001C080E02A9600
:101EC0000FB6F894DEBF0FBECDBFDF91CF911F914B
:101ED0000F91FF90EF90DF90CF90BF90AF909F90C9
:101EE0008F907F906F905F9008950E94DA0E0E940D
:101EF000841A0E94D01D81110E94860E0E947514C2
:101F00000C94E003CF93DF930E94AC10EC01811599
:101F100021E5920708F045C0811530E5930708F0E8
:101F200094C0883E910528F5803E910508F0F8C0E0
:101F3000883A910570F4853A910508F07CC08130AB
:101F4000910509F475C008F4E8C0049708F0E8C0EA
:101F5000E4C08F3B910508F0E0C0C85AD0E0CC0F38
:101F6000DD1FCA58DE4F0990D881C02DCE01946480
:101F7000D8C0811540E2940758F4811551E09507C7
:101F800008F0CEC08D3E910508F4C7C09065C9C069
:101F9000C11580E4D80708F4C0C0DF70CE01906A94
:101FA000C0C0811525E59207A8F4811534E5930793
:101FB00008F095C0811543E5940708F07BC08115B2
:101FC00052E5950708F061C0D82FCC27CE01816F6C
:101FD000906AA7C0C11589E5D807A0F4C11528E506
:101FE000D20708F082C0C11536E5D30708F095C0C6
:101FF0008C2F0E9440118F7190E0D82FCC27CE01FA
:1020000090628FC0C1154AE5D40708F474C0CE01B0
:1020100090568115904208F080C08D2F8F710E94DC
:102020004011DD27D0628F71AE01582BCA0179C0F3
:1020300081E090E076C0C55AD0E0CC55DE4F888173
:10204000C82FD0E0CE0190646CC074E0969587955F
:102050007A95E1F7282F23703C2F337081E090E0D0
:1020600002C0880F991F3A95E2F79C68AC01522B89
:102070009A019C2F9F709695969550E2959FE0014E
:102080001124C9018C2B9D2B4CC08370992721E012
:1020900030E002C0220F331F8A95E2F79C2F9695FD
:1020A000969580E2989FE0011124C22BD32BCE019C
:1020B0009C6837C08370992721E030E002C0220F6E
:1020C000331F8A95E2F79C2F9695969540E2949F50
:1020D000E0011124C22BD32BCE019A6822C0D82F45
:1020E000CC27CE01846F906A1CC0DC2FCC27CE0198
:1020F000806F906A16C08C2F8F700E94401194E000
:10210000D695C7959A95E1F7CF70D0E0DC2FCC2714
:10211000D0699E01282BC90104C080E090E001C075
:10212000CE01DF91CF9108952CE2829FC00111244E
:10213000FC012BE0729FE00DF11D1124E60FF11D53
:10214000EE0FFF1FE852FF4F8591949108950E9472
:1021500094100E94820F08958238910569F1B0F4BD
:102160008133910509F46DC048F48932910509F471
:1021700063C08A32910509F469C0089585339105D9
:1021800009F455C089339105B9F00895833E91054E
:1021900069F138F4803E9105B1F0823E910509F174
:1021A0000895863E9105A9F1873E9105B9F1843ED7
:1021B000910509F064C023C02091FB0220FD4FC0AF
:1021C00021FD4DC008958091FB0280FD44C08091A7
:1021D000FC0280FF44C08091FB0284FD42C083EE7C
:1021E0004DC08091FB0282FF38C0F5CF8091FB0289
:1021F00082FD33C08091FC0280FD31C0ECCF809124
:10220000FC0281FF32C08091FB0284FD2AC087EE70
:1022100035C08091FB0283FF26C0F5CF8091FB0281
:1022200083FD21C08091FC0281FD1FC0ECCF809115
:10223000FB0285FD1CC01DC08091FB0285FD19C0FD
:1022400016C08091FB0286FD16C017C08091FB026C
:1022500086FD13C010C089E311C082EE0FC080EE6E
:102260000DC080E00BC086EE09C084EE07C089E295
:1022700005C085E303C08AE201C081E390E00895D0
:102280009091FB0292FF0DC0282F2871283019F47D
:10229000877F846006C0282F2471243011F48B7F3F
:1022A000886093FF0DC0282F2871283119F4877E8C
:1022B000846106C0282F2471243111F48B7E88613B
:1022C0002091FC0220FF0DC0382F3871383019F4EE
:1022D000877F816006C0382F3171313011F48E7FD5
:1022E000886021FF0DC0282F2871283119F4877EBE
:1022F000816106C0282F2171213111F48E7E886101
:1023000094FD877E089580E008950C94BE0D0E9490
:1023100097128FE39CE90197F1F700C000000E943B
:10232000971280E00E94C11180FF04C00E948511B5
:102330000C94742108950C9487110E94C40D81118E
:1023400002C00E946C0E0E94CF0D8093AA020E94D0
:10235000D70D9093FC028093FB020E949B110E9478
:10236000D30D682F70E080E090E00E94E00760915C
:1023700012027091130280911402909115020C9434
:102380001808E82FF0E0EE0FFF1FEB5FFC4F808195
:1023900091810895089580EA8A95F1F7089500C023
:1023A00008950C94CB1108950C94D3110C94D4116E
:1023B0000C94D3110C94D811F894E82FE295EF7097
:1023C000F0E031A1282F2F7081E090E001C0880F4C
:1023D0002A95EAF7982F9095932391A392A1892BA0
:1023E00082A3789408950F931F93CF93DF93C2EB4A
:1023F000D1E089918F3F11F00E94DC1181E0C63B52
:10240000D807B9F7C7EAD1E002EB11E089918F3F15
:1024100011F00E94DC110C171D07C1F7DF91CF915D
:102420001F910F910895BF92CF92DF92EF92FF928A
:102430000F931F93CF93DF938C01C62FD0E0CE0173
:102440008E549E4F6C01FC0190819F3F09F450C057
:10245000B62EF894E92FE295EF70F0E081A19F701D
:1024600021E030E001C0220F9A95EAF7822B81A388
:1024700082A12095282322A378940E94CF11E7EA15
:10248000F1E042EB51E021E030E0E12CF12C6191F0
:102490006F3F89F0A62FA295AF70B0E090968C9117
:1024A00090E06F7002C0959587956A95E2F780FD80
:1024B00002C0C90102C080E090E0E82AF92A220F98
:1024C000331F4E175F0719F7F60180818F3F11F018
:1024D0000E94DC1161E0E114F10409F460E08B2D4D
:1024E0000E94D111CC0FDD1FC00FD11FF982E882ED
:1024F000DF91CF911F910F91FF90EF90DF90CF90E0
:10250000BF9008950E94F31188E0E5E0F3E0DF0159
:10251000982F1D929A95E9F7EDEFF2E0DF011D92F9
:102520008A95E9F784E00E94E2120C945303FF922B
:102530000F931F93CF93DF93CDB7DEB728970FB6D6
:10254000F894DEBF0FBECDBF8E010F5F1F4F88E036
:10255000F80111928A95E9F7F12C6F2DC8010E94BC
:102560001312F394F4E0FF12F8CF48E050E0B80102
:102570008DEF92E00E942129FF24F394009709F443
:10258000F12C892B41F088E0F801ADEFB2E0019029
:102590000D928A95E1F72F2D44E065E073E08DEF11
:1025A00092E00E94E3120E9455038F2D28960FB6E9
:1025B000F894DEBF0FBECDBFDF91CF911F910F9179
:1025C000FF9008950895FF920F931F93CF93DF9389
:1025D000F82E092F162FD72FC42F222349F081E080
:1025E0008093AD020E9427219093AC028093AB02AE
:1025F0008091AD028823D9F08091AB029091AC021A
:102600000E943F21059798F0EF2DF02FA12FBD2FAD
:1026100080E090E04C2F50E08417950734F421912E
:1026200031912D933D930196F7CF1092AD02DF913A
:10263000CF911F910F91FF9008950E943F230E9418
:10264000C30E0C944B230E944F230E94750F0C94D1
:1026500069230E94C5200E9426230E94B10E0E9479
:102660001D130E9423130E94BB0EFBCF80912401F7
:1026700090E0880F991FFC01E45EFE4F2081FC0171
:10268000E45FFE4F80819091B402191614F42093F8
:10269000B4029091B40297FF04C0922F9195909349
:1026A000B4029091B502191614F42093B5029091DA
:1026B000B50297FF03C021952093B5029091B70210
:1026C000191614F48093B7029091B70297FF04C0D3
:1026D000982F91959093B7029091B602191614F421
:1026E0008093B6029091B60297FF03C081958093C4
:1026F000B6023091B4023323E1F02091B5022223D7
:10270000C1F045EB3403C0011124992319F09093D3
:10271000B40203C081E08093B40235EB2303C0010F
:102720001124992319F09093B50203C081E080939E
:10273000B5024091B702442379F03091B6023323B9
:1027400059F025EB4203A00111245093B702320344
:10275000C00111249093B602089540912401242FC2
:1027600030E0220F331FF901E45EFE4F90818D3E71
:1027700011F4919502C08E3E19F49093B5023EC0BB
:102780008F3E11F4919502C0803F19F49093B402EA
:1027900035C0F901E45FFE4F9081893F19F08A3F0F
:1027A00021F491959093B60229C08B3F11F4919535
:1027B00002C08C3F19F49093B70220C09FE0980F9D
:1027C000983078F421E030E0B90102C0660F771F3D
:1027D0009A95E2F7CB019091B302892B8093B302D3
:1027E0000DC08D3F11F481E007C08E3F11F482E0EF
:1027F00003C08F3F19F483E080932401809124016A
:1028000048130C94361308958D3E39F49091B50217
:1028100097FF39C01092B50208958E3E29F4909129
:10282000B5021916BCF32FC08F3E39F49091B40253
:1028300097FF29C01092B4020895803F29F4909127
:10284000B4021916BCF31FC0893F39F49091B60247
:102850001916CCF41092B60208958A3F29F490918B
:10286000B60297FF10C0F6CF8B3F39F49091B702B4
:1028700097FF09C01092B70208958C3F21F4909100
:10288000B7021916BCF39FE0980F983078F421E056
:1028900030E0A90102C0440F551F9A95E2F7CA0122
:1028A00080959091B30289238093B30208950E948A
:1028B00027212091B402211104C02091B5022223C6
:1028C00021F09093B1028093B0022091B6022111C1
:1028D00004C02091B702222321F09093AF0280938D
:1028E000AE0282EB92E00C94931FEF92FF920F9353
:1028F0001F93CF93DF9300D000D000D0CDB7DEB7C9
:1029000086E0E2EBF2E0DE01119601900D928A95ED
:10291000E1F7E090B402F090B5020091B602109198
:10292000B7021092B4021092B5021092B602109241
:10293000B702E11002C0FF20B1F08091B002909187
:10294000B1020E943F21E0912401F0E0EE0FFF1F51
:10295000EC5EFE4F208131812817390720F4E09288
:10296000B402F092B502111102C00023B1F08091BF
:10297000AE029091AF020E943F21E0912401F0E06D
:10298000EE0FFF1FEC5FFE4F2081318128173907C2
:1029900020F40093B6021093B7028091B402811123
:1029A0000BC08091B502811107C08091B6028111E0
:1029B00003C08091B70281110E945714EB82FC8200
:1029C0000D831E8386E0FE013196A2EBB2E00190FA
:1029D0000D928A95E1F726960FB6F894DEBF0FBEEA
:1029E000CDBFDF91CF911F910F91FF90EF90089590
:1029F000E2EBF2E086E0DF011D928A95E9F70895A7
:102A0000EF92FF920F931F93CF93DF938B01682F69
:102A100011110AC0442329F0E82FF0E0E950FD4FDE
:102A20006491762F862F75C0212F30E0E82FF0E0DB
:102A3000442321F0E950FD4FE491F0E046E0049F8B
:102A4000C0011124CFEFD0E0BE010E9487284BEADD
:102A50004603C001479F900D1124800F911D800FE8
:102A6000911D982F990F890FAE01421B530B4E9F5A
:102A7000D0014F9FB00D5E9FB00D11249B2F189F6A
:102A8000A0011124452F55278E01041B150B0E9F05
:102A9000A0010F9F500D1E9F500D11247E01E81ABA
:102AA000F108E29E8001E39E100DF29E100D1124AC
:102AB000212F3327C21BD30BCE9F9001CF9F300D08
:102AC000DE9F300D112462307105A9F048F46115C4
:102AD000710569F061307105C9F48B2F752F0DC038
:102AE0006430710581F058F06630710579F47E2FFD
:102AF0008B2F932F0DC0832F7B2F9E2F09C08E2FDE
:102B00007B2F952F05C08E2F732F02C07E2F852F10
:102B1000692FDF91CF911F910F91FF90EF90089552
:102B200041E00E940015089508950E9490150895AF
:102B3000CF93DF93762FE901682F842F0E9495159C
:102B4000798368838A83DF91CF91089580910D0303
:102B5000282F269530E02115310519F48170826007
:102B600005C02532310524F08170886480930D03FF
:102B7000089588E090E00C943629CF92DF92EF928E
:102B8000FF926B017C010E94A615B701A60188E0A7
:102B900090E0FF90EF90DF90CF900C945429EDE0FF
:102BA000F3E083E0808311828FEF8283838314823A
:102BB00060817181828193810C94BD1580910D0398
:102BC00080FF02C08695089580E0089590911103DA
:102BD000933018F49F5F90931103882351F0609114
:102BE0000D0370910E0380910F03909110030C94CC
:102BF000BD15089581E00C94E61590911103992379
:102C000019F0915090931103882351F060910D03B6
:102C100070910E0380910F03909110030C94BD15D9
:102C2000089581E00C94FD1570E00C94011C6091F6
:102C3000290180910D0380FF0AC08091280123E0C3
:102C4000829FC00111248E5E9C4F0C9414168091BB
:102C50002A0190912B01891780F7E82FF0E09F015E
:102C6000220F331FE20FF31FEE5EFC4F1182108222
:102C700012828F5FF0CF90910D0390FF16C090915C
:102C80002A0120912B01921770F4E92FF0E0DF0167
:102C9000AA0FBB1FEA0FFB1FEE5EFC4F8183608310
:102CA00042839F5FF0CF0C9417160895CF93DF9364
:102CB00000D01F92CDB7DEB790910D0390FF0AC0F0
:102CC0009E012F5F3F4F0E9498154B8169818A8139
:102CD0000E943B160F900F900F90DF91CF910895B7
:102CE000CF93DF93EC01EC81F0E0EE50FE4F449186
:102CF000EDE0F3E0628181810E9456168C818F5F46
:102D00008C83DF91CF910895CF93DF93EC01EDE0B9
:102D1000F3E0438162818C810E9456168C818F5F23
:102D20008C83DF91CF9108950F931F93CF93DF93FF
:102D300000D01F92CDB7DEB78C018091B80281110F
:102D40000AC09E012F5F3F4F4FEF6FEF0E94981513
:102D50008A818093B802F8018481813051F028F093
:102D6000823061F44091B8020AC08091B80240E01C
:102D700007C06091B80240E080E003C040E080E01E
:102D800060E00E943B16F801848190E0019663E0C8
:102D900070E00E949B2884830F900F900F90DF912A
:102DA000CF911F910F910895AF92BF92CF92DF9272
:102DB000EF92FF920F931F93CF93DF9300D01F9258
:102DC000CDB7DEB7182FF62E042FE22E90910D030B
:102DD00090FF6DC0E92FE695AE2FB0E0AA54BE4F2C
:102DE0008C918093C2029E7F923061F49E012F5F8E
:102DF0003F4F812F0E9498154B8169818A810E94E3
:102E00003B1643C0823019F4009110033EC0863057
:102E100019F410910E0339C08930D9F38931A9F51D
:102E2000E9518E2F8170D82EE695F0E0EE50FD4FDF
:102E3000A590B490C12CBB2460912C01C61618F546
:102E40002C2D30E0A29EC001A39E900DB29E900D4D
:102E5000112470E00E948728812FD11002C0860FB4
:102E600001C0861B90912A01290F311DA901440F31
:102E7000551F240F351F2E5E3C4F402F6F2D0E9493
:102E80009815C394D9CF0E94171610930E03F09291
:102E90000F0300931003EE2051F060910D03709129
:102EA0000E0380910F03909110030E94BD150F90A7
:102EB0000F900F90DF91CF911F910F91FF90EF90A6
:102EC000DF90CF90BF90AF900895EDE0F3E0918157
:102ED000282F4381628188E0890F0C94D41681E009
:102EE0000C946517EDE0F3E09181282F4381628116
:102EF00088EF890F0C94D41681E00C947217EDE0E2
:102F0000F3E0628121E1620F08F46FEF282F438123
:102F100081810C94D41681E00C947F17EDE0F3E0EE
:102F2000628121E1621B08F460E0282F43818181E6
:102F30000C94D41681E00C948E17EDE0F3E04381FD
:102F400021E1420F08F44FEF282F628181810C9418
:102F5000D41681E00C949D17EDE0F3E0438121E16C
:102F6000421B08F440E0282F628181810C94D41622
:102F700081E00C94AC1720E00C94D416FF920F93D0
:102F80001F93CF93DF93EC01F12C0FEF10E06091D2
:102F90002C01F616F0F480912A012F2D30E0280F35
:102FA000311DC901880F991F280F391F2E5E3C4F14
:102FB00070E0C8010E949B28962F8C8140911003DD
:102FC00060910F03F99E800D11240E949815F394CF
:102FD000DECF0E9417169A818C8190FF02C08F5F0E
:102FE00001C081508C83DF91CF911F910F91FF9091
:102FF0000895AF92BF92CF92DF92EF92FF920F931C
:103000001F93CF93DF93FC01828180FF02C00FEFFB
:1030100001C001E010E043E1A42E80912C011817BB
:1030200008F043C080912A01C12ED12CE601C80FBF
:10303000D11DCE01880F991FC80FD91FCE5EDC4F5E
:10304000198218821A8234E0E32EF12CB12C80917F
:10305000BA028B0D84312CF06A2D0E947928892FB9
:1030600005C087FF03C090912C01890F082E000C2A
:10307000990BC816D90691F4809110038E9DA0017A
:103080008F9D500D112455954795559547959E0157
:1030900060910F0380910E030E949815B00EF1E02D
:1030A000EF1AF108A1F61F5FB8CF0E9417168091A2
:1030B000BA02013031F4811102C080912C0181509B
:1030C00007C090E0019660912C0170E00E949B285F
:1030D0008093BA02DF91CF911F910F91FF90EF90F3
:1030E000DF90CF90BF90AF900895CF9380912A0149
:1030F00090912B01891770F4E82FF0E09F01220FC7
:10310000331FE20FF31FEE5EFC4F1182108212821A
:103110008F5FF0CFC0E060912C01C617C0F5EC2F97
:10312000F0E070E0CF010E949B2820912A01820FDD
:103130002091B902022E000C330B90E0E217F30746
:10314000CCF020912701022E000C330B2E173F07E5
:103150008CF09C01220F331F820F931F9C012E5E67
:103160003C4F4091100360910F0380910E030E9429
:1031700098150BC0FC01EE0FFF1F8E0F9F1FFC0167
:10318000EE5EFC4F118210821282CF5FC4CF0E948C
:103190001716209126018091B902820F8093B902FF
:1031A00090912701920F9093270119165CF4082E35
:1031B000000C990B40912C0150E0415051098417AB
:1031C00095071CF0219520932601CF9108958F92A9
:1031D0009F92AF92BF92CF92DF92EF92FF920F93A6
:1031E0001F93CF93DF938C01FC014481C42FD0E067
:1031F0009E01DE010E94DF289B01AC010E94F528A0
:103200006B017C01E0E2F0E0EC1BFD0BA5E5B0E01A
:103210009B01AC010E94F5284B015C019F01DF017D
:103220000E94D7289B01AC010E9400299B01AC01A0
:103230002C0D3D1D4E1D5F1DC501B4010E94AF2820
:10324000C22FD22F2A3228F4F3E02F9F90011124AD
:103250000DC025E530E02C1B3109C901880F991FED
:10326000280F391F37FF02C02F5F3F4F3595279535
:10327000C22FC095F12C85E5E82EED1A80912C0126
:10328000F816C8F4F1FC02C08E2D01C08D2F90916C
:103290002A012F2D30E0290F311DA901440F551FA0
:1032A000240F351F2E5E3C4F4C2F60910F030E9460
:1032B0009815F394E3CF0E941716F80184818111C9
:1032C00002C091E003C0803219F49FEF9093250172
:1032D00090912501890FF8018483DF91CF911F918F
:1032E0000F91FF90EF90DF90CF90BF90AF909F90A5
:1032F0008F9008950F931F93CF93DF93EC0100E01D
:1033000010E080912C01282F30E00217130724F5DC
:1033100090912A019801290F311DA901440F551FD1
:10332000240F351F2E5E3C4F869590E04C81081788
:1033300019071CF4442331F002C0411103C040912D
:10334000100301C040E060910F0380910E030E94C2
:1033500098150F5F1F4FD5CF0E9417168C8190E0F4
:103360000196817099278C83DF91CF911F910F91E6
:103370000895EDE0F3E080818E7F8083608171812C
:10338000828193810E94BD151092C3022FEF80E7C6
:1033900092E0215080409040E1F700C000000C9482
:1033A000171660910D03669570E04BE050E08DE2DA
:1033B00091E00E941429892B19F481E08093C302C3
:1033C0000E9427219093BC028093BB0208959091A4
:1033D0000D0390FF35C09170811102C0926006C04C
:1033E000853210F0986402C0880F982B90930D03DB
:1033F000662351F060910D0370910E0380910F03CD
:10340000909110030E94BD1560910D03669570E0C8
:103410004BE050E08DE291E00E941429892B19F0D5
:103420001092C30202C00E94D11981E08093BE02B3
:103430004091100360910F0380910E030C94BB1711
:103440000895682F90910D03969581E0890F85323C
:1034500008F081E00C94E71981E00C94211A682FA0
:1034600090910D0396958FEF890F09F484E20C94E7
:10347000E71981E00C942F1A61E00C94E719EDE054
:10348000F3E080818160808386950C943C1A809162
:103490000D0380FD0C94B9190C943F1A60E00C9454
:1034A000E7198091C10281112EC00E94C40D8111C3
:1034B00004C00E946C0E0E94CF150E94B915609343
:1034C0000D0370930E0380930F03909310036E7F90
:1034D00061F40E94CF150E94B91560930D0370939B
:1034E0000E0380930F03909310030E94A615109271
:1034F000C30280910D0380FF03C086950E944E1A7F
:1035000081E08093C10208950F931F93CF93DF93BF
:103510008091C302882309F485C08091C202E091A2
:103520000D03E695E81BE093BD02823049F4F0E01C
:10353000E251FE4FE491CE2FD0E000E716E149C002
:10354000863049F4F0E0E551FE4FE491CE2FD0E013
:1035500004E816E13EC0893051F4E695F0E0E85108
:10356000FE4FE491CE2FD0E00EEB17E132C08F304A
:1035700051F4E695F0E0EB51FE4FE491CE2FD0E010
:1035800009EF17E126C0853149F4F0E0EE51FE4F16
:10359000E491CE2FD0E005E718E11BC0883181F01F
:1035A000833239F4E0EEF1E0C591D49104E916E1FB
:1035B00010C0843251F4C4EFD1E00AE719E109C028
:1035C000C8E2D0E007EE18E104C0C0EDD7E004E99E
:1035D00015E18091BE02882361F01092BE020E9424
:1035E00027219093BC028093BB021092C0021092DC
:1035F000BF020E942721E091BB02F091BC028E1B0A
:103600009F0B8F3F9F4770F4EC0FFD1FF093BC02A0
:10361000E093BB028BEB92E0F801DF91CF911F9119
:103620000F910994DF91CF911F910F9108958823F5
:1036300011F0FA0101C0FB010994CF93DF93C82F69
:10364000D62F0E94DE158C1740F00E94DE158D17D4
:1036500020F4DF91CF910C942C1A8C2FDF91CF9115
:103660000C943C1A1F93CF93DF93FB01128111112D
:10367000C3C0EC010E94DB0C8272CD3CFCE5DF078D
:1036800009F49AC0A8F5C73CECE5DE0709F476C05A
:10369000A8F4C43C9CE5D90709F45FC028F4C33CF6
:1036A000DC4509F457C054C0C53C9CE5D90709F472
:1036B00059C0C63CDC4509F45CC04AC0CA3CFCE5C4
:1036C000DF0709F46AC050F4C83CECE5DE0709F4F2
:1036D0005AC0C93CDC4509F45BC03AC0CB3C9CE510
:1036E000D90709F45FC0CC3CDC4509F460C030C0A8
:1036F000C23DFCE5DF0709F46FC088F4CF3C9CE5D0
:10370000D90709F460C008F45CC0C03DFCE5DF07E0
:1037100009F45CC0C13DDC4509F45BC019C0C53D7E
:103720009CE5D90709F460C050F4C33DFCE5DF0710
:1037300009F455C0C43DDC4509F454C009C0C63D78
:103740009CE5D90709F455C0CE35DD4509F454C0D0
:1037500011E052C00E94471A4FC049E35AE16CE29F
:103760007AE104C04CE25AE169E37AE10E94171B56
:1037700043C04CE757E16FE677E1F8CF4FE657E1FA
:103780006CE777E1F3CF4AE957E16BE877E1EECFF9
:103790004BE857E16AE977E1E9CF48EB57E169EA9D
:1037A00077E1E4CF49EA57E168EB77E1DFCF41E128
:1037B00056E16AEF75E1DACF4AEF55E161E176E172
:1037C000D5CF81E017C065E082E010C068E086E0F8
:1037D0000DC06EE089E00AC064E18FE007C067E1D8
:1037E00085E104C088E106C062E289E10E941D1BF8
:1037F00003C083E20E943C1A812FDF91CF911F9179
:103800000895519A2BB12D7F3BB132604FB7F89498
:10381000FC01CB01880F991F680F791F6E0F7F1F66
:10382000E617F70789F0819198E03BB9000000C0E6
:1038300087FF2BB9880F000000C000C000C02BB963
:1038400000C09A9591F7ECCF4FBF8FE594E00197B8
:10385000F1F700C000000895CF93DF93EC01FB0166
:103860008281882309F43CC1C430FDE5DF0760F4A0
:10387000CB3F9CE5D90788F49E0122503C4524317A
:10388000310508F02EC109C0C236EDE5DE0729F08A
:10389000C63AFDE5DF0709F024C10E94D70D9093D9
:1038A000FC028093FB02C1318CE5D80709F4C6C045
:1038B00008F042C0C930ECE5DE0709F49BC000F512
:1038C000C5308CE5D80709F485C078F4C330ECE541
:1038D000DE0709F478C008F07AC0C230DC4509F090
:1038E000F5C08091FB028160EFC0C7309CE5D9072D
:1038F00009F478C008F07AC08091FB028061E4C0CE
:10390000CD30FCE5DF0709F487C058F4CB309CE5E7
:10391000D90709F479C008F07BC08091FB02886068
:103920006FC0CF30FCE5DF0709F480C008F082C02B
:103930008091FB02877FC8C0CE3F9CE5D90709F480
:1039400071C000F5C531FCE5DF0709F485C068F4F6
:10395000C3319CE5D90709F475C008F095C00E94F1
:1039600088078091FB028F77AFC0CC3FFCE5DF0773
:10397000A9F108F054C0CB3FDC4509F0A7C0809105
:10398000FC0240C0C230EDE5DE0709F489C058F4FE
:10399000C1158DE5D80709F45AC008F069C08091B7
:1039A000FC0282602FC0C236EDE5DE0709F47CC060
:1039B000C63AFDE5DF0709F481C0C330DD4509F0F3
:1039C00085C080E06EC08091FB0282607DC08091E6
:1039D000FB0216C08091FB02886076C08091FC02D9
:1039E00082604FC08091FB0280626EC08091FB02BA
:1039F00080646AC00E9488078091FB02806864C06E
:103A0000846062C081603DC08091FB028E7F5CC09B
:103A10008091FB028D7F58C08091FB0216C080917F
:103A2000FC0218C08091FC028D7F2BC08091FB02AC
:103A30008F7E4AC08091FB028F7D46C08091FB0241
:103A40008F7B42C08091FB02877F8B7F3DC080913E
:103A5000FC028D7F8E7F15C08091FB0282FB2227A6
:103A600020F991E0922790FB82F990FB83F92CC01A
:103A70008091FC02982F909591708E7F892B90FBFE
:103A800081F98093FC0222C00E9488078091FB028A
:103A900087FB222720F991E0922790FB87F914C039
:103AA00081E00E946E0E12C08091FB0284FB2227EF
:103AB00020F991E0922790FB84F906C08091FB02E7
:103AC000982F909590FB80F98093FB028091FB02E8
:103AD0009091FC020E94E80D0E94880780E001C0DE
:103AE00081E0DF91CF9108958FE891E00197F1F7A0
:103AF00000C0000008950C94EE02CF93DF93ADEE6A
:103B0000B1E0CBEED1E021E030E071E0AF3EB707AD
:103B100059F18D91E82FE295EF70F0E041A18F709F
:103B2000B90102C0660F771F8A95E2F7CB01962F85
:103B30009095942391A392A1892B82A38991E82F38
:103B4000E295EF70F0E041A18F70B90102C0660FFD
:103B5000771F8A95E2F7CB01962F9095942391A336
:103B600092A1892B82A3D1CF0E94741D83B182FBC5
:103B7000882780F9199902C090E001C092E0892B52
:103B80008093C8028FB1829581707D9902C090E0C8
:103B900001C092E0892B8093C902DF91CF910895F3
:103BA0004F925F926F927F928F929F92AF92BF924D
:103BB000CF92DF92EF92FF920F931F93CF93DF93F9
:103BC00008EC12E08DEEC82E81E0D82E9BEEE92E97
:103BD00091E0F92E26EC822E22E0922EC4ECD2E067
:103BE0005801512C412C33E0632E712CD501ED91FD
:103BF0005D014E2F440F440FF60121916F01E22F1A
:103C0000E295EF70F0E080A190E02F7002C09595F2
:103C100087952A95E2F781709927D7015D917D01FB
:103C2000E52FE295EF70F0E020A130E05F7002C078
:103C3000359527955A95E2F7F901E170FF2720FFA6
:103C400002C0E2E0F0E0E82BF92BE42BD801ED9381
:103C50008D01EF70F0E0E552FE4F9081F40180811C
:103C6000890F808383304CF088818F5F888360E088
:103C7000852D0E947B1D21E001C020E0D4018C91A4
:103C80008E3F44F488818150888361E0852D0E94B5
:103C90007B1D21E0F4018081082E000C990BB301FB
:103CA0000E949B28D4018D934D01422A5394219662
:103CB000B2E05B129BCF842DDF91CF911F910F91CA
:103CC000FF90EF90DF90CF90BF90AF909F908F903C
:103CD0007F906F905F904F900895CF93DF938631E0
:103CE0009C4541F5EB010E94DB0C982F8A812091C5
:103CF000020130910301882379F09A7A81E009F476
:103D000080E08093CA02911102C069E201C065E3BC
:103D1000C9010E9463200AC08091CA02811102C0B9
:103D200069E201C065E3C9010E946E200E941D0D79
:103D300080E001C081E0DF91CF9108950F931F9340
:103D4000CF93DF93C42FD22FFC0182818823C9F047
:103D50004093CD020E9427219093CC028093CB0206
:103D600080E28C0F883008F057C0C77081E001C036
:103D7000880FCA95EAF7DF91CF911F910F910C94AC
:103D8000E5048091CD02481330C08091CB02909120
:103D9000CC020E943F21883C910538F510E21D0FAE
:103DA000CD17B9F080E28C0F883040F4C77081E005
:103DB00001C0880FCA95EAF70E94EC04183028F574
:103DC00081E09D2F977001C0880F9A95EAF70E94B5
:103DD000E504802F0E94DC041830F0F4D77081E0F5
:103DE00001C0880FDA95EAF70AC080E28C0F8830AC
:103DF00098F4C77081E001C0880FCA95EAF7DF9197
:103E0000CF911F910F910C94EC04802FDF91CF91F3
:103E10001F910F910C94DC04DF91CF911F910F91B2
:103E200008950F939C01CB01243F4CE5340731F1F9
:103E300088F4293DFCE53F07D9F02A3D4CE53407DD
:103E400079F1283D3C45A9F506E221EE41EE68ED09
:103E50007CE52BC0263FFCE53F07E1F0A8F0273FBB
:103E60003C4539F507E225EE46EE67EF7CE51DC0DF
:103E700007E225EE45EE69ED7CE517C006E221EE8E
:103E800040EE64EF7CE511C007E225EE44EE65EFFD
:103E90007CE50BC006E221EE42EE66EF7CE505C054
:103EA00008E221E045EE6AED7CE50E949E1E80E07E
:103EB00008C0FC018281882319F01092CD0201C054
:103EC00081E00F9108959093F1018093F00108959E
:103ED0009093D3028093D2020895E091D202F091A0
:103EE000D302309721F00190F081E02D099480E019
:103EF0000895E091D202F091D302309799F0209189
:103F00004401222359F02091FB0227FF07C0DC0166
:103F10002C9111962C93119726E02C930280F3811B
:103F2000E02D09940895E091D202F091D3023097E8
:103F300039F022E0DC012C930480F581E02D099416
:103F400008952091D0023091D1022817390771F0DD
:103F50009093D1028093D002E091D202F091D302EB
:103F6000309721F00680F781E02D09940895209183
:103F7000CE023091CF022817390771F09093CF020B
:103F80008093CE02E091D202F091D302309721F0DB
:103F90000084F185E02D09940895FC01329680910A
:103FA0004401882331F08091FB0287FF02C09EE12B
:103FB00001C096E080E0915028F021912223D9F3AE
:103FC0008F5FF9CF0895662351F120914401222398
:103FD000E9F02091FB0227FF19C0462F4695469530
:103FE00046954E31E0F4677021E030E002C0220FC8
:103FF000331F6A95E2F7FC01E40FF11D828190E026
:104000002823392381E0232B69F409C0FC0132966F
:1040100008962191621729F0E817F907D1F780E097
:10402000089581E008959C01FC0132969FEF80E0A5
:104030004191461789F09F3F19F4411101C0982F13
:104040008F5F8630A9F79F3F39F0F901E90FF11D25
:1040500097FDFA956283089508959C012A5F3F4F6A
:10406000FC014281461301C0128201968217930718
:10407000B9F70895262F2695269526952E3168F4B2
:10408000FC01E20FF11D677021E030E001C0220F5A
:104090006A95EAF78281282B22830895262F269598
:1040A000269526952E3170F4FC01E20FF11D677004
:1040B00021E030E001C0220F6A95EAF72095828165
:1040C00028232283089520914401222329F020915E
:1040D000FB0227FD0C943A200C94132020914401FC
:1040E000222329F02091FB0227FD0C944E200C94F2
:1040F0002D2020914401FC013296222331F0809141
:10410000FB0287FF02C08EE101C086E0DF011D9245
:104110008A95E9F7089508950C948B2083E08093A5
:10412000D4020C948C20811102C081E001C082E095
:104130008093D4020C948C200C94932081E0809383
:10414000D4020C948C200C949E2008950C94A520ED
:104150000C94A6200C94A5200C94A5200C94A520CA
:10416000CF930E94AC200E9497120E94AA20C0E028
:104170008C2F0E94C111892B29F4CF5FC430C1F765
:1041800080E001C081E0CF91089508951F920F92C1
:104190000FB60F9211248F939F93AF93BF9380918B
:1041A000D502811113C080914B0390914C03A091D3
:1041B0004D03B0914E034196A11DB11D80934B0359
:1041C00090934C03A0934D03B0934E03BF91AF91D6
:1041D0009F918F910F900FBE0F901F901895809117
:1041E0005303843031F10E94C0031092D50220E4C1
:1041F00088E190E00FB6F894A895809360000FBE18
:104200002093600083B7817F846083BF83B7816020
:1042100083BF7894889583B78E7F83BF0FB6F89459
:10422000A895809160008861809360001092600082
:104230000FBE08950E9488070C94C40382E084BDD9
:1042400093E095BD9AEF97BD80936E0008952FB7C8
:10425000F89480914B0390914C03A0914D03B09141
:104260004E032FBF08952FB7F89460914B037091C0
:104270004C0380914D0390914E032FBF08959C01F4
:104280004FB7F89480914B0390914C03A0914D034C
:10429000B0914E034FBF821B930B089578941F92E9
:1042A0000F920FB60F9211248F939F93AF93BF93EA
:1042B00080914B0390914C03A0914D03B0914E031C
:1042C0000196A11DB11D80934B0390934C03A093C5
:1042D0004D03B0934E03BF91AF919F918F910F907B
:1042E0000FBE0F901F90189581E08093E00080E250
:1042F0008093D8001092C9008FE19EE40197F1F7F6
:1043000000C0000087E090EBDC0180935C03909399
:104310005D03A0935E03B0935F039CE088E10FB65A
:10432000F894A895809360000FBE90936000FFCF33
:104330008091F9020895089522E02093E9002FEF7B
:104340003091E800215035FD06C035ED3A95F1F782
:1043500000002111F5CF2091E80025FF0BC040E0BF
:1043600050E066E070E00E94DB238091E8008E77E9
:104370008093E8000895CF93DF9320914401222396
:1043800039F02091FB0227FF03C060E222E002C067
:1043900068E021E02093E9002FEF3091E800215000
:1043A00035FD06C035ED3A95F1F700002111F5CF46
:1043B0002091E80025FF1DC0EC018091440181118E
:1043C00005C040E050E068E070E003C070E040E00D
:1043D00050E0CE010E94DB238091E8008E7780932D
:1043E000E80080E2FE01A9EDB2E001900D928A950D
:1043F000E1F7DF91CF9108958093D6027093D802B0
:104400006093D70280915303843001F582E080935A
:10441000E9008FEF9091E800815095FD06C095ED81
:104420009A95F1F700008111F5CF8091E80085FFA2
:104430000DC040E050E063E070E086ED92E00E9445
:10444000DB238091E8008E778093E8000895BC011B
:1044500084E00C94FC21BC0183E00C94FC2180914D
:104460005203811109C00E946C250E94C9258091C8
:10447000E20084608093E200089510925203089550
:104480000C94A32060914F0381E0611101C080E092
:104490000C948E209091530381E0943009F080E0D9
:1044A00060914F030C94932042E061EC81E00E9404
:1044B000E52442E261EC82E00E94E52490915303FE
:1044C00081E0943009F080E060914F030C949C20CF
:1044D00080915503833009F461C030F4813071F06C
:1044E000823009F49AC008958A3009F486C08B306E
:1044F00009F46CC0893009F0A8C020C08091540331
:10450000813A09F0A2C08091E800877F8093E8009B
:104510008091580390915903892B21F460E289ED31
:1045200092E003C060E080E090E070E00E9426240A
:104530008091E8008B778093E80008958091540380
:10454000813209F082C080915803909159030297FB
:1045500008F07BC08091E800877F8093E80080911D
:10456000E80082FD05C0809153038111F8CF6DC032
:104570002091F3008091F20090E0922B029731F4A9
:104580008091F100813011F0863021F48091F100AA
:104590008093F9028091E8008B7753C08091540397
:1045A000813A09F052C08091580390915903892BA8
:1045B00009F04BC08091E800877F8093E8008091EC
:1045C000E80080FFFCCF8091440136C08091540305
:1045D0008132D9F58091580390915903892BA9F51F
:1045E0008091E800877F8093E8000E941A258091DF
:1045F0005603809344010C948807809154038132C0
:1046000021F58091E800877F8093E8000E941A25B9
:10461000809157038093FA02089580915403813A60
:10462000A1F48091E800877F8093E8008091E80002
:1046300080FFFCCF8091FA028093F1008091E80026
:104640008E778093E8000C941A25089584B7877FAD
:1046500084BF0FB6F894A89580916000886180931C
:104660006000109260000FBE90E080E80FB6F894F2
:1046700080936100909361000FBE0C949E200E9475
:104680006C250E94C925E2EEF0E080818460808381
:1046900078940C945E2888E391E00C94681F8091D4
:1046A00053038530A9F480915303853079F40E9437
:1046B000EF20809151038823B1F30E94B02088231A
:1046C00091F30E94C5230E948807EDCF0C941A2114
:1046D000089508950C946C23292F33272330310536
:1046E000C9F060F42130310581F02230310509F044
:1046F00044C08BE390E025E234E043C02132310531
:10470000E1F02232310549F138C082E190E020E643
:1047100034E037C099278130910549F028F002979D
:1047200061F5E7EFF3E005C0E1E2F4E002C0E7E0A5
:10473000F4E0849190E09F0124C06115710541F07F
:1047400061307105D1F489E090E020E534E019C0D2
:1047500089E090E027E334E014C06115710541F071
:104760006130710551F486EB90E022E734E009C036
:1047700080E490E028E235E004C080E090E020E0B2
:1047800030E0FA0131832083089580E189BD82E120
:1047900089BD09B400FEFDCF8091D8008F7D809344
:1047A000D8008091E00082608093E0008091E0007A
:1047B00081FDFCCF0895CF92DF92EF92FF920F938D
:1047C0001F93CF93DF93EC018B017A010E9439256F
:1047D000811133C0E114F10439F0F7018081918136
:1047E000081B190BC80FD91FC12CD12C011511059D
:1047F00019F18091E80085FD16C08091E8008E7760
:104800008093E800E114F10449F0F701808191817F
:10481000C80ED91ED182C08285E00FC00E94392502
:10482000882321F30AC089918093F1000150110976
:10483000FFEFCF1ADF0ADACF80E0DF91CF911F912F
:104840000F91FF90EF90DF90CF90089520915A0341
:1048500030915B032617370748F06115710539F46D
:104860002091E8002E772093E80001C0B901FC01F7
:1048700020E06115710579F1809153038823F1F1EE
:104880008530F1F18091E80083FD3CC08091E80023
:1048900082FD2EC08091E80080FFEBCF2091F300D5
:1048A0008091F20090E0922B6115710551F08830F3
:1048B000910538F421912093F1006150710901961E
:1048C000F3CF21E0089709F020E08091E8008E778F
:1048D0008093E800CECF2111CFCF0AC0809153033F
:1048E000882361F0853061F08091E80083FD0AC083
:1048F0008091E80082FFF2CF80E0089582E0089581
:1049000083E0089581E0089520915A0330915B037C
:104910002617370748F06115710539F42091E80032
:104920002E772093E80001C0B901FC0120E0611559
:10493000710591F180915303882309F440C08530BB
:1049400009F43FC08091E80083FD3DC08091E800FC
:1049500082FD2FC08091E80080FFE9CF2091F30015
:104960008091F20090E0922B6115710559F088302A
:10497000910540F424912093F10031966150710922
:104980000196F2CF21E0089709F020E08091E8003D
:104990008E778093E800CBCF2111CCCF0AC08091D5
:1049A0005303882361F0853061F08091E80083FD36
:1049B0000AC08091E80082FFF2CF80E0089582E093
:1049C000089583E0089581E00895982F973068F561
:1049D0009093E900981739F07091EC002091ED0068
:1049E0005091F00003C0242F762F50E021FD02C02B
:1049F0009F5FECCF3091EB003E7F3093EB00309126
:104A0000ED003D7F3093ED003091EB00316030934D
:104A1000EB007093EC002093ED005093F000209198
:104A2000EE0027FDE5CF80E008958F708093E900C8
:104A300081E008958091540387FF11C08091E800C0
:104A400082FD05C0809153038111F8CF11C0809180
:104A5000E8008B770BC080915303882349F0809145
:104A6000E80080FFF8CF8091E8008E778093E8001F
:104A700008952091E4003091E50095E64091EC0026
:104A8000842F817040FF23C08091E80080FD1DC00D
:104A900080915303882399F0853099F08091EB0041
:104AA00085FD11C04091E4005091E50024173507C1
:104AB00029F3915011F09A01E1CF84E0089582E04A
:104AC000089583E0089581E0089580E0089540917D
:104AD000E80042FFDDCF08950E94DA250E94E2251A
:104AE000E0EEF0E0808181608083E8EDF0E080819D
:104AF0008F77808319BCA7EDB0E08C918E7F8C936B
:104B000080818F7E80831092520308950F931F93AC
:104B1000CF93DF930E94DA250E94E225C8EDD0E012
:104B200088818F77888388818068888388818F7D5A
:104B3000888319BC1092530310924F0310925103B3
:104B40001092500300EE10E0F80180818B7F80838B
:104B500088818160888342E060E080E00E94E524F3
:104B6000E1EEF0E080818E7F8083E2EEF0E08081F4
:104B700081608083808188608083F80180818E7F5E
:104B80008083888180618883DF91CF911F910F910D
:104B90000895E8EDF0E080818F7E8083E7EDF0E01E
:104BA00080818160808384E082BF81E080935203B2
:104BB0000C948625E8EDF0E080818E7F8083109252
:104BC000E20008951092DA001092E10008951F9219
:104BD0000F920FB60F9211242F933F934F935F9331
:104BE0006F937F938F939F93AF93BF93EF93FF93B5
:104BF0008091E10082FF0BC08091E20082FF07C03C
:104C00008091E1008B7F8093E1000E945D2880917C
:104C1000DA0080FF1FC08091D80080FF1BC0809108
:104C2000DA008E7F8093DA008091D90080FF0DC07A
:104C300080E189BD82E189BD09B400FEFDCF81E03C
:104C4000809353030E942F2205C019BC1092530376
:104C50000E943D228091E10080FF19C08091E20016
:104C600080FF15C08091E2008E7F8093E2008091EA
:104C7000E20080618093E2008091D800806280939E
:104C8000D80019BC85E0809353030E944222809192
:104C9000E10084FF30C08091E20084FF2CC080E1FD
:104CA00089BD82E189BD09B400FEFDCF8091D800A5
:104CB0008F7D8093D8008091E1008F7E8093E1000A
:104CC0008091E2008F7E8093E2008091E20081601B
:104CD0008093E20080914F03882311F084E007C0A5
:104CE0008091E30087FD02C081E001C083E08093F2
:104CF00053030E944A228091E10083FF29C08091E2
:104D0000E20083FF25C08091E100877F8093E1006E
:104D100082E08093530310924F038091E1008E7FD5
:104D20008093E1008091E2008E7F8093E200809189
:104D3000E20080618093E20042E060E080E00E9457
:104D4000E5248091F00088608093F0000E9440226A
:104D5000FF91EF91BF91AF919F918F917F916F9153
:104D60005F914F913F912F910F900FBE0F901F9029
:104D700018951F920F920FB60F9211242F933F9305
:104D80004F935F936F937F938F939F93AF93BF9353
:104D9000CF93DF93EF93FF93C091E900CF708091A1
:104DA000EC00D82FD17080FDD0E81092E9008091FE
:104DB000F000877F8093F00078940E94FD26109287
:104DC000E9008091F00088608093F000CD2BCF70D7
:104DD000C093E900FF91EF91DF91CF91BF91AF9127
:104DE0009F918F917F916F915F914F913F912F9103
:104DF0000F900FBE0F901F9018951F93CF93DF93C6
:104E0000CDB7DEB7AA970FB6F894DEBF0FBECDBF01
:104E1000E4E5F3E08091F100819323E0EC35F207C3
:104E2000C9F70E9468228091E80083FF2EC180911B
:104E3000540390915503492F50E04A30510508F032
:104E400024C1FA01EE59FF4F0C94D128803821F08B
:104E5000823809F01AC108C0809150039091510323
:104E6000992389F082600FC0809158038F7087303A
:104E700008F00BC18093E9008091EB0085FB882747
:104E800080F91092E9009091E800977F9093E800F4
:104E90008093F1001092F100D1C0282F2D7F09F0EE
:104EA000F4C0882319F0823061F0EFC0809156037E
:104EB000813009F0EAC0933009F080E0809351031B
:104EC0002EC08091560381112AC0809158038F70A3
:104ED0002FEF280F263008F0D8C08093E9002091EA
:104EE000EB0020FF1CC0933021F48091EB00806226
:104EF00014C09091EB0090619093EB0021E030E0C2
:104F0000A90102C0440F551F8A95E2F74093EA00B9
:104F10001092EA008091EB0088608093EB00109281
:104F2000E9008091E800877F8093E8000E941A25BD
:104F3000ACC08111AAC0109156031F778091E30085
:104F40008078812B8093E3008091E800877F8093B5
:104F5000E8000E941A258091E80080FFFCCF809134
:104F6000E30080688093E300111102C082E001C079
:104F700083E08093530389C08058823008F085C055
:104F800080915603909157038C3D53E0950779F536
:104F900083E08A838AE289834FB7F894DE0113960F
:104FA00020E03EE051E2E32FF0E050935700E4911F
:104FB00020FF03C0E295EF703F5FEF708E2F90E00F
:104FC000EA3010F0C79601C0C0968D939D932F5F75
:104FD000243149F74FBF8091E800877F8093E80034
:104FE0006AE270E0CE0101960E94262416C060910C
:104FF000580370915903AE014F5F5F4F0E946A23BF
:10500000BC01892B09F441C09091E800977F9093EF
:10501000E80089819A810E9484248091E8008B773E
:105020008093E80032C0803881F58091E800877F66
:105030008093E80080914F038093F1008091E80015
:105040008E7772CF811121C08091560390915703C2
:1050500099270297D4F48091E800877F8093E80035
:105060008091560380934F030E941A2580914F032D
:10507000811106C08091E30087FD02C081E001C07C
:1050800084E0809353030E9454228091E80083FFC0
:105090000AC08091E800877F8093E8008091EB0050
:1050A00080628093EB00AA960FB6F894DEBF0FBE25
:1050B000CDBFDF91CF911F9108950895CF93809137
:1050C00053038823A1F0C091E900CF709091EC00C8
:1050D000892F817090FD80E8C82B1092E9008091A3
:1050E000E80083FD0E94FD26CF70C093E900CF91B8
:1050F000089587FB082E062687FD819567FD61953B
:105100000E9408290EF4919507FC81950895AA1B29
:10511000BB1B51E107C0AA1FBB1FA617B70710F0A2
:10512000A61BB70B881F991F5A95A9F780959095D4
:10513000BC01CD01089597FB072E16F4009407D00B
:1051400077FD09D00E94872807FC05D03EF4909592
:1051500081959F4F0895709561957F4F0895A1E2C5
:105160001A2EAA1BBB1BFD010DC0AA1FBB1FEE1FE1
:10517000FF1FA217B307E407F50720F0A21BB30B2C
:10518000E40BF50B661F771F881F991F1A9469F7A8
:1051900060957095809590959B01AC01BD01CF0104
:1051A0000895EE0FFF1F0590F491E02D09940E94E1
:1051B000DF28332312F48A1B9B0B0C94F028A29F48
:1051C000B001B39FC001A39F700D811D1124911DDB
:1051D000B29F700D811D1124911D08950E94DF283A
:1051E000B7FF0895821B930B08950E94DF28A59FA7
:1051F000900DB49F900DA49F800D911D11240895D2
:10520000B7FF0C94F5280E94F528821B930B089594
:10521000991B79E004C0991F961708F0961B881F08
:105220007A95C9F780950895FC014150504030F0BF
:1052300001900616D1F73197CF0108958827992755
:105240000895FB01DC0104C08D910190801921F4C7
:1052500041505040C8F7881B990B0895F999FECF2B
:1052600092BD81BDF89A992780B50895A6E1B0E076
:1052700044E050E00C946829A8E1B0E042E050E03E
:105280000C946829262FF999FECF92BD81BDF89A1A
:10529000019700B4021639F01FBA20BD0FB6F8947A
:1052A000FA9AF99A0FBE08950396272F0E94432970
:1052B0000E944229252F0E944329242F0C94432920
:1052C0000196272F0E9443290C944229DC01CB012F
:1052D000FC01F999FECF06C0F2BDE1BDF89A319606
:1052E00000B40D9241505040B8F70895F894FFCFA4
:1052F000C800740228006801780014000100010051
:10530000010001001000200010001000100001003A
:105310000400200002010102001300131301191AF6
:105320001B1C1D1E1F2021229821BB219C212B22EA
:1053300027229B2101E200E900EA00B500B600B790
:1053400000CD008301CC008A019201940121022347
:105350000224022502260227022A02B300B4006FAB
:10536000007000818283E200E900EA00B500B60027
:10537000B700CD008301CC008A0192019401210283
:10538000230224022502260227022A02B300B400C7
:105390006F00700081828333949697343536666748
:1053A000F7F6929395F00001020202020606060942
:1053B00009090909090F0F0F0F0F0F1515151819F6
:1053C000191919191919191919232400FF010001B4
:1053D0000000FFFF0000010001FF0031F532F40082
:00000001FF
